:10000000F92B00308A000408840A82070034523435
:1000100048342034203420343D34203430343034DB
:100020002E3430343034203425342034203400341D
:10003000543465346D34703420343D3420343034DD
:1000400030342E34303430342034433420342034AF
:1000500000346E346F342034723465347334703449
:100060002E34663472346F346D3420344434483462
:100070005434003443346834653463346B3473343B
:1000800075346D3420344534723472340034543451
:1000900069346D34653420346F34753474342134EC
:0200A00000342A
:1000A40064008001840A04060319003404065328FA
:1000B40034308312AD00F130AC00AC0B5F28AD0BD3
:1000C4005F286428080006308312AE001330AD00A8
:1000D400AD30AC00AC0B6C28AD0B6C28AE0B6C28AF
:1000E40073280800831206153430AD00F130AC00DB
:1000F400AC0B7A28AD0B7A287F28831206110000F6
:1001040000000800B2003203031D8B283108803E32
:10011400FC20023083123206031D08003108C03E61
:10012400FC2008001A308312AC00AC0B97280000A6
:100134008312051808003530AC00AC0B9F288312DD
:10014400051C08002130AC00AC0BA62801300800C7
:10015400831605100510831205104130AD00EE30F2
:10016400AC00AC0BB328AD0BB3280000831205140C
:100174001330AC00AC0BBC28BF2883160514080050
:100184008312B100B00130083107AF002F0884009A
:10019400831300080319080030083107AF002F0843
:1001A4008400000827210130AF002F08B007103069
:1001B400300203180800C528AE002C088400012072
:1001C400003A0319F7282C0884000120AD002E08FA
:1001D40084002D08831380000130AD002D08AC0786
:1001E4000130AD002D08AE07DF282E0884008313EC
:1001F400800108008312B0005A20831206100611F1
:100204000F30AE002E088605000083123008F03946
:10021400AE002E0886045A2074200F308312AE00DC
:100224002E088605000083123008AE000330031048
:10023400AE0DFF3E031D192903102E0DF039AF003A
:100244002F0886045A2074200800AE00061400000B
:10025400831206110F30AC002C0886052E08F039E5
:10026400AC002C08860406150330AD009730AC00B2
:10027400AC0B3A29AD0B3A293F29831206110F30F2
:10028400AC002C0886052E08AC0003300310AC0D1E
:10029400FF3E031D482903102C0DF039AD002D0835
:1002A400860406150000831206110800340835047C
:1002B40003198529B901B90AB51B6C29013003104A
:1002C400B40DB50DFF3E031D61290130B800380897
:1002D400B9075E2935083702031D7229340836022E
:1002E400031C7A293408B6023508031CB703B70285
:1002F40001300310B50CB40CFF3E031D7B29013003
:10030400B902031D6C293708B5003608B40008008B
:10031400B101B2012C082D040319C129B301B30A98
:10032400AD1BA02901300310AC0DAD0DFF3E031D24
:1003340095290130B0003008B30792290130031029
:10034400B10DB20DFF3E031DA1292D082F02031D7F
:10035400AD292C082E02031CB6292C08AE022D0848
:10036400031CAF03AF02311401300310AD0CAC0C0D
:10037400FF3E031DB7290130B302031DA029320833
:10038400AD003108AC0008005A20831606080F3966
:10039400860000000F308312B100310886055A2010
:1003A4008316061086100611831286100610061195
:1003B4005A20831206080F398600000083120608AB
:1003C4003038860074205A200F308312B10031086F
:1003D40086053030B1003108860474205A200F306D
:1003E4008312B10031088605000030308312B10059
:1003F4003108860474205A200F308312B10031086A
:10040400860500008312861674205A202830FC20AA
:100414000630FC200C30FC205A208312851508007D
:100424008312AE019901B001AF0183120518262A87
:100434000130AC002C08AF0765302F02031C242ABE
:100444009901990A252A172A1330AC00AC0B282AE3
:100454002B2A831205183F2A0130AC003008073CD0
:10046400013E362A0310AC0DFF3E031D342A2C082E
:10047400FF3AAD002D08AE055E2A0130AC0030080D
:10048400073C013E472A0310AC0DFF3E031D452ADD
:100494002C08AD002D08AE04AF018312051C5E2AA2
:1004A4000130AC002C08AF0765302F02031C5C2A16
:1004B4009901990A5D2A4F2A0130AC002C08B00733
:1004C40008303002031C162A2E080800013085006B
:1004D40001308316850086018312850183168511F8
:1004E4008312851183160510831292019301120859
:1004F4001A3E84008001013092070318930A0030E9
:10050400930700301302113003191202031C792AD5
:1005140002308316810015308312BC004B30BB00BF
:10052400BE30BA00BA0B942ABB0B942ABC0B942A93
:100534000000C6211530BC004B30BB00BE30BA00F1
:10054400BA0BA22ABB0BA22ABC0BA22A000065206C
:10055400AA209420003A0319BE2B1222BA003A08AA
:1005640096001222BA003A0895001222BA003A08FC
:1005740098001222BA003A0897001222BA003A08E8
:10058400940019080319C82A4130C02B150816070E
:10059400BA0018083A07BB0017083B071406031DE6
:1005A400B62B1608BA00BB013A088C003B088D0034
:1005B4001508BA00BB010C08BD00BC013A083C0494
:1005C4008C003B083D048D001808BA00BB013A08B2
:1005D4008E003B088F001708BA00BB010E08BD004F
:1005E400BC013A083C048E003B083D048F00803077
:1005F4000F02013003190E02031C0B2B2D30BA001D
:100604003A08A000FF300E058E007F300F058F00E2
:10061400112B1230BA003A08AC001A30DE200A302E
:10062400B4000030B5006430AC000030AD000F08F9
:10063400AF000E08AE008A212D08B7002C08B600C2
:1006440058213408303EBA003A08A1000A30B400F8
:100654000030B5000A30AC000030AD000F08AF0028
:100664000E08AE008A212D08B7002C08B6005821C8
:100674003408303EBA003A08A2000A30B400003010
:10068400B5000F08B7000E08B60058213408303EF4
:10069400BA003A08A400DF30BA003A08A500433093
:1006A400BA003A08A6002030BA003A08A700203061
:1006B400BA003A08A800A901B101013084201A3017
:1006C400C2200130BA003A08AC001A30DE200A30E9
:1006D400B4000030B5006430AC000030AD000D084B
:1006E400AF000C08AE008A212D08B7002C08B60014
:1006F40058213408303EBA003A08A1000A30B40048
:100704000030B5000A30AC000030AD000D08AF0079
:100714000C08AE008A212D08B7002C08B600582119
:100724003408303EBA003A08A2000A30B40000305F
:10073400B5000D08B7000C08B60058213408303E47
:10074400BA003A08A4002530BA003A08A5002030BF
:10075400BA003A08A6002030BA003A08A600A90157
:10076400B10102308420C52B0130FC208312B10179
:10077400013084203430BF2B23308312BA003A086E
:10078400AC001A30DE201A30C22085159201930184
:10079400831285110330BC000830BB007730BA00E7
:1007A400BA0BD22BBB0BD22BBC0BD22B83128515CD
:1007B4000330BC000830BB007730BA00BA0BE02B22
:1007C400BB0BE02BBC0BE02B013083129207031808
:1007D400930A003093071308803ACF0080304F0209
:1007E400031DF62B063012020318A92ACA2B831301
:0C07F4000C3084002C3052208301682A55
:02400E00F93F78
:00000001FF
